:020000040800F2
:10000000700700209D010008A5010008A701000855
:10001000A9010008AB010008AD01000800000000C4
:10002000000000000000000000000000AF01000818
:10003000B101000800000000B3010008B50100088C
:10004000B7010008B7010008B7010008B7010008B0
:10005000B7010008B7010008B7010008B7010008A0
:10006000B7010008B7010008B7010008B701000890
:10007000B7010008B7010008B7010008B701000880
:10008000B7010008B7010008B7010008B701000870
:10009000B7010008B7010008B7010008B701000860
:1000A000B7010008B7010008B7010008B701000850
:1000B000B7010008B7010008B7010008B701000840
:1000C000B7010008B7010008B7010008B701000830
:1000D000B7010008B7010008B7010008B701000820
:1000E000B7010008B7010008B701000800F002F8E6
:1000F00000F044F80AA090E8000C82448344AAF17E
:100100000107DA4501D100F039F8AFF2090EBAE87B
:100110000F0013F0010F18BFFB1A43F0010318473B
:10012000880D0000A80D0000103A24BF78C878C1DF
:10013000FAD8520724BF30C830C144BF04680C60ED
:10014000704700000023002400250026103A28BF35
:1001500078C1FBD8520728BF30C148BF0B60704739
:10016000002070471FB59DE8030000F0C9FB00F0B8
:10017000A7F81FBD10B500F00CF910BD00F06FF925
:100180001146FFF7EFFF00F079FE00F05FFB03B4CC
:10019000FFF7F0FF03BC00F045FD00000948804771
:1001A00009480047FEE7FEE7FEE7FEE7FEE7FEE759
:1001B000FEE7FEE7FEE7FEE704480549054A064B71
:1001C00070470000110E0008ED00000870010020CB
:1001D0007007002070030020700300200FB4044952
:1001E00010B503AA029800F03DF810BC5DF814FBAE
:1001F000640000202DE9F0410E46044600202062F4
:100200002046E168884730B3252805D0D4E901218C
:100210009047206A401CF2E7E168204600278847A3
:10022000050018D0A5F14100192802D820354FF457
:1002300000673246294620462760FFF791FF40B10C
:10024000012804D0F61D26F007060836D8E7361D2B
:10025000D6E72846DAE7206ABDE8F08170477047A4
:1002600070470000074B70B50D467B4400F011F855
:100270000446284600F020F810B14FF0FF3070BD62
:10028000204670BDF30B000001694A1C026108782A
:10029000704700B58FB0CDE90131002105910549C6
:1002A0007944CDE9031011466846FFF7A3FF0FB06C
:1002B00000BD0000E5FFFFFF007B00F080007047FD
:1002C00010B54248542100F0D1FA4148542100F0C1
:1002D000CDFA4048542100F0C9FA3F493B483C4A16
:1002E0003F4B08603D490A603A491960531C036559
:1002F000481C1065012008653B48344A39A1784400
:1003000000F008FA20B9384878440A3800F0A7FA13
:1003100037482F4A35A1784400F0FCF920B9344819
:1003200078440A3800F09BFA32482A4A2FA17844D0
:1003300000F0F0F920B92F4878440A3800F08FFA1D
:1003400040232248DC000021224600F0BFF920B102
:1003500025487844543800F082FA1D48224640234C
:10036000002100F0B3F920B121487844543800F05E
:1003700076FA184822461023002100F0A7F9002839
:1003800006D01C487844BDE81040563800F067BAE3
:1003900010BD104870B5006D20F001040B4800F04E
:1003A0002FFA0B4800F02CFA0A4800F029FA09E06D
:1003B000206D20F00105204600F022FA204600F0D2
:1003C00073F82C46002CF3D170BD00001000002003
:1003D00064000020B8000020040000200800002075
:1003E0000C000020720000008A0B00007700000063
:1003F000760B0000620B00000EB5CDE9000100F0A5
:10040000F1FB029069460120ABBE0EBD08B56946FE
:1004100000900220ABBE08BD1FB58DE807006946FD
:100420000520ABBE04B010BD1FB58DE80F006946B6
:100430000620ABBEF6E708B5694600900920ABBEC2
:1004400008BD1CB5CDE9000169460A20ABBE1CBD44
:10045000704708B5694600900C20ABBE08BD7546D4
:1004600000F02CFAAE4605006946534620F007001E
:10047000854618B020B5FFF79FFEBDE820404FF03D
:1004800000064FF000074FF000084FF0000B21F07E
:100490000701AC46ACE8C009ACE8C009ACE8C0094B
:1004A000ACE8C0098D46704770B50446051F00F0E2
:1004B0000BFA0068002C14BF446870BD002C18BFF4
:1004C000AC423CBF20466468F8D301680A18AA42CF
:1004D00018BF456003D12A680546114401602868A9
:1004E0004119A1421CBF6C6070BD616869602168E0
:1004F0000844286070BD2DE9F04705460C46C868E1
:1005000020F4201040F48000C860800602D5084620
:1005100000F027FBE06841F282014FF0FF39014013
:10052000022903D0204600F0C5FAB5E000F42041CE
:10053000B1F5004F0FD1C00306D56168E06A88426B
:1005400000D80846606006E02069E062606060698B
:10055000FFF77FFFA061A0680022EEB200280DDA4D
:10056000E1688B050AD4C043A06041F4903022605A
:10057000E0606068411C61600670A5E0E06890463C
:10058000226040F40050E060206968BB6069FFF7BA
:1005900052FF012704F12405A0B1A08910F4407F87
:1005A00008D0E06900F0DBF9206118B1E06840F4A0
:1005B000006016E0E7612561E06820F4407040F4D7
:1005C00080600EE0E06900F0CAF900282061F1D0F7
:1005D000E06840F4006010F4407FE06002D140F435
:1005E0008070E06020696060E06825696FF0010A52
:1005F000C1051FD56168E06A884200D80846411BE2
:1006000004D02246284600F05FFAF0BBE068010201
:1006100003D5E562C4E9015854E0691CE1626160F8
:10062000E16940F48030491EC4E9021030462E7062
:10063000BDE8F087010202D500F480320AE060686C
:10064000411C61600670E0680A2E40F48030E06072
:1006500006D00022E16A6068814203D90B4602E0BD
:100660000122F7E70346A7895B1B7F0503D4E769EF
:100670009F4200DDE2B1814200D80146E5620F1AD7
:10068000C4E90158002B09DD00E005E022461946C7
:10069000284600F019FA08B14846C9E747B1A069F1
:1006A000E5626560C01BA061E06840F01000E0609A
:1006B000E068000208D56168A069E562491B08444A
:1006C0006560A0615046B3E73046B1E770B5C468D5
:1006D000A50713D0650211D4B2F5807F09D0B2F519
:1006E000007F06D0B2F5806F08D1012300F124010C
:1006F00006E05D1E6FF07F46B54201D3012070BD5C
:100700000161C361416024F470611143C160002044
:1007100070BD00002DE9F0410C4607461646104614
:1007200000F06EF82078611C61280AD0722802D08F
:1007300077283CD102E00125002405E002250424AD
:1007400002E0082448F2020511F8010B2B2806D01C
:10075000622809D011F8010C74280AD00BE045F08A
:10076000030544F00204EFE745F0040544F00104FA
:10077000EAE744F0100438462146FFF73DFE411CED
:1007800015D00021316171604FF40071F560F161A5
:100790007061200704D530460222002100F00EF9D6
:1007A000306D40F0010030653046BDE8F08100203A
:1007B000FBE72DE9F0410D460646104C206DC107C0
:1007C00004D0410804D020F00104F7E722460EE0EF
:1007D000542000F0C4F807000ED0206D47F001014E
:1007E000084354212065384600F040F83A4629462F
:1007F0003046BDE8F0418DE70020D6E7100000202C
:100800002DE9F04704464FF000094FF0FF37C56867
:10081000D4E90486A80707D0204600F07FF93046C7
:10082000FFF7F4FD002802DA3846BDE8F087280516
:1008300002D54046FFF738FE4C21204600F016F85E
:10084000206D20F0010020654846EEE710B5044613
:10085000AFF300802046BDE81040FFF798BC10B50C
:1008600000F0A6F9BDE8104000F09CB94FF000027E
:1008700000B5134694469646203922BFA0E80C5096
:10088000A0E80C50B1F12001BFF4F7AF090728BF71
:10089000A0E80C5048BF0CC05DF804EB890028BFED
:1008A00040F8042B08BF704748BF20F8022B11F016
:1008B000804F18BF00F8012B7047000000487047B8
:1008C0000C01002070470000004870471401002010
:1008D000704770477047704738B504460A46002095
:1008E0006946AFF30080002808BF38BD0246009972
:1008F000204600F0A4F9012038BD012000F0F3B932
:10090000F8B5AFF30080054600200C46102000BF6C
:100910000646A819A0420DD9324669460020AFF319
:100920000080070008BF00F0DEF90098A04218BF61
:100930000546C419FFF7C8FF05600746F01D20F003
:1009400007004619284600F073F9B44208BFF8BD05
:10095000A21B31463868BDE8F84000F070B970B5A8
:100960000646FFF7B1FF056806F10B0020F007040B
:10097000B4429CBF002070BD2B466A68BAB11068B3
:10098000A04210D304F1080188423CBF506858606F
:1009900007D35168101941601168091B0160586044
:1009A0001460101D70BD13465268002AE7D121461D
:1009B0002846FFF791FF0028DED170BD2DE9F041F8
:1009C000044616460D464769007B80072ED0384600
:1009D000FFF731FD50BB3EB3012E02D0022E25D1D0
:1009E00004E0204600F045F905441DE03846FFF7D5
:1009F00030FDE168002841F01001E16005DA204691
:100A000000F058F80120BDE8F081C9030BD56268F9
:100A1000E16A914200D81146A26911442269891AFB
:100A2000814200DD08460544002D01DA0220EAE794
:100A3000E16A6068E268814206D29103E06203D510
:100A400022F4003141F01002A6690027AE4213DC07
:100A5000E16A814201D90B4600E0034603EB060C34
:100A60002369ACEB030CAC4506DD814201D98C4611
:100A700000E084469C4505D1A760276042F0200035
:100A8000A5620DE0AD1BE669AE1B8142A66000D9F0
:100A90000846C01A281A20605819606022F0200009
:100AA00003490840E060002084F84870ABE700008C
:100AB000BFCFD7FFC16821F4001141F08001C160B0
:100AC00000218160016070472DE9F047814614469E
:100AD0000E464FF0FF383248D5685769054209D0B5
:100AE0003846A169FFF7ADFC002811DB2C48C04354
:100AF0000540E5602B46324649463846FFF78CFCF8
:100B0000A16920F00042B21A11440028A16103D06B
:100B10002046FFF7CFFF4046BDE8F08770B504469A
:100B20000569C06A6168884200D80846E16821F416
:100B30002011E160C90312D5A84208D02246411B0A
:100B40002846FFF7C1FF10B14FF0FF3070BD002005
:100B5000E562C4E90150E06820F48030E0600020E4
:100B600070BD10B50446C06820F02000E060A16AA6
:100B7000A06988420DD02046FFF7D0FFE06820F43E
:100B8000405040F01000E060A06AA0612069E0627F
:100B9000606044F24001E0688843E06010BD0000FE
:100BA00010000200002801D000F03CB8704700009F
:100BB00010B5014602A000F07DF8012010BD000034
:100BC00053494752545245443A205265646972650C
:100BD00063743A2063616E2774206F70656E3A20EB
:100BE0000000000010B5431C02E010F8011B71B1B9
:100BF0008107FAD14FF0013202C88C1A8C4314EAF3
:100C0000C211F9D0C01A0A0603D0C01E10BDC01A06
:100C100010BD0A0401D0801E10BD0902FCD0401E88
:100C200010BD000001491820ABBEFEE726000200FF
:100C300000210160C0E90110704710207047034691
:100C400040688C46002818BF88423CBF0346406875
:100C5000F8D318681844884207D00CF1030020F03C
:100C60000700001D411A521A0146081D0A60FFF7CD
:100C70001BBC10B50146C268900703D0900607D58B
:100C8000886A0AE000F03EF801210160881E10BD6C
:100C90008B69486818440B69C01A91F848301BB139
:100CA00091F84910401A10BD1103FCD50028FADD57
:100CB000401E10BD70B505460C460A2000E06D1CB4
:100CC00000F018F835B128780028F8D102E0641C4B
:100CD00000F010F814B120780028F8D1BDE8704079
:100CE0000A2000F007B810B500F010F8BDE8104079
:100CF000FFF758BF08B569468DF800000320ABBE6A
:100D000008BD0000004870470C01002010B5012804
:100D100005D0002103A0FFF7CDFF012010BD09A1E0
:100D2000F8E7000053494752544D454D3A204F755E
:100D300074206F662068656170206D656D6F7279D3
:100D4000000000003A2048656170206D656D6F728B
:100D50007920636F7272757074656400AFF3008000
:100D60000CB50022019200922748016841F48031BD
:100D700001604FF4A063016801F400310091019912
:100D8000491C0191009911B901999942F3D1016867
:100D9000890302D50121009100E000920099012908
:100DA00030D11A490A6842F010020A600A6822F03B
:100DB00007020A600A6842F002020A604168416064
:100DC00041684160416841F480614160416821F4BB
:100DD0007C114160416841F4E8114160016841F0D3
:100DE0008071016001688901FCD5416821F003012F
:100DF0004160416841F0020141604168C1F38101F5
:100E00000229FAD10CBD000000100240002002406F
:100E100010B50F48016841F00101016041680D4AB9
:100E20001140416001680C4A11400160016821F4E1
:100E300080210160416821F4FE0141604FF41F01EF
:100E40008160FFF78BFF05494FF00060086010BD1F
:100E5000001002400000FFF8FFFFF6FE08ED00E082
:100E60008A68002A01DCFFF746BB521E8A604A6886
:100E7000C0B2531C4B6010707047000002480068FD
:100E8000FFF7ACF9FEE70000000000203A747400A0
:100E90003A7474003A74740048656C6C6F20776F14
:100EA000726C642100000000C80E000800000020E1
:100EB0001000000028010008D80E000810000020D3
:100EC0006007000044010008980E000800000000C0
:080ED00000000000000000001A
:04000005080000ED02
:00000001FF
